:1000000083128501860105289B29831685018601B7
:10001000061481160113831286147A2294019030FB
:100020008B008A22940803191228523014060319EF
:100030005F21493014060319832131301406031956
:10004000051430301406031905105830140603192E
:100050002E21503014060319812054301406031940
:100060003D204830140603193C21940156224F309C
:100070006A224B306A22562212280F11B0203130EA
:100080006A220F193E28080056221030A6001030B0
:10009000A5005F2056222030A6001030A5005F206A
:1000A00056223030A6001030A5005F205622403086
:1000B000A6001030A5005F205622940108002608F3
:1000C000840000081D22A60AA50B5F2808002E0840
:1000D000FF3A0319AD0AAE0A0800AD01AE010800EF
:1000E00027082D06031D792828082E06031D7928C8
:1000F00008000630B521672070280310A70CA80C53
:1001000008009401AB0194080319832843301406B6
:100110000319E328503014068F14AE216D20B0204F
:100120000F1DAE2870203130A4000230B521240804
:10013000840000089C00A40A2408840000089D0094
:10014000C4210830B5218422A40A67200630B521D5
:10015000AC03AC0B952831306A228F28B3210800FC
:1001600023303B222308AC0027303B220230A30778
:1001700028303B223030A4003B22A40A2408A30BE1
:10018000BC28B0080319CB28B003031D132AB10FF4
:10019000132A0F110800AB012C08A300AB07270896
:1001A000AB072808AB073130A400A30A2408840059
:1001B0000008AB07A40AA30BD628AB08031D132A1B
:1001C0000F157D2008009401B020AE210030B5212C
:1001D000C421842231089C0032089D000230B521E0
:1001E000C4210830B52184220630B52133089C0093
:1001F00034089D000230B521C4210830B521842285
:100200000630B52135089C0036089D000230B52126
:10021000C4210830B52184220630B52137089C005E
:1002200038089D000230B521C4210830B521842250
:100230000630B5210630B5210630B5210630B5218E
:1002400039089C003A089D000230B521C4210830CD
:10025000B5218422B32131306A220800AE21023058
:10026000B521FF309C009D00C4210930B521183014
:10027000B5218422B3210800AE210030B521FF3022
:100280009C009D00C4210630B5210630B521063002
:10029000B5210630B5210630B5210630B52106302E
:1002A000B5210130B5210730B5210830B5218422B0
:1002B00084220130B5210730B521B3210800273051
:1002C0003B2228303B22A901AA0156220130A8076F
:1002D0000318A70AAE210430B521EB211D081D2209
:1002E0001C081D220630B5210130AA070318A90AEF
:1002F00027082906031D6B2928082A06031D6B29D8
:100300000F15B3210800AE2100309D0000309C0085
:100310000030B521C42184220830A0000430B5216A
:10032000EB211D081D221C081D220630B521A00B43
:100330008E29B32108009900030E9A00061EA229F7
:100340000612A32906165B22243014060319442042
:100350008B101A0E83009A0E1A0E09008501842252
:10036000051485140800850108009E0006309B00D6
:1003700003109E0C031CBE298515C02985110000A1
:10038000E3219B0BB82908008511E32108309B006D
:1003900003109C0C031CCE298515D0298511000063
:1003A000E3219B0BC82906309B0003109D0C031C06
:1003B000DB298515DD2985110000E3219B0BD5295B
:1003C0008511E32108000515000000000000000071
:1003D0000000051108008316851583120000E32133
:1003E00008309B0005150000851DF8290314F92924
:1003F00003109C0C05119B0BF22906309B00051580
:100400000000851D052A0314062A031005119D0C02
:100410009B0BFF2903109D0C9D0CE3218316851176
:100420008312851108008B13B321861644200030F7
:10043000A7004030A80063211C2AA100210E0F391B
:10044000093C031C272A210E0F39303E2A2A210E8F
:100450000F39573E6A2221080F39093C031C342A00
:1004600021080F39303E372A21080F39573E6A22BA
:1004700020306A22080094018400940803193D2A60
:100480004A22800094080319422A800EF0394A2239
:10049000800708001408403C031C512A1408D03E71
:1004A000542A1408DF39C93E940108000D306A222D
:1004B0000A306A220800083098007F2206180800D7
:1004C0007A220618652A0310662A0314940C980BE6
:1004D000602A080093000830970086107A220310E3
:1004E000930C031C752A8614762A86107A22970BA1
:1004F0006F2A86141F309500950B7C2A08000F3058
:100500009600960B812A080064309F007A229F0B88
:10051000862A0800562248306A226F306A226C30E0
:100520006A226C306A2269306A2265306A2273302E
:100530006A2220306A2250306A2269306A2263308F
:100540006A2250306A2272306A226F306A22673023
:100550006A2220306A2276306A2231306A222E30B6
:100560006A2230306A2234306A22562252306A229D
:100570007C306A2244306A227C306A2250306A22FF
:100580007C306A2231306A227C306A2230306A2222
:100590003F306A2256220800562250306A227C30B0
:1005A0006A2243306A227C306A2244306A227C30DC
:0E05B0006A2245306A223F306A225622080035
:084000000500020001000000B0
:02400E00F13F80
:00000001FF
